:0500000002003341C6BF
:02000B0041C7EB
:02001300617E0C
:02001B00617F03
:020023006180FA
:02002B006181F1
:10003300759840758780758921758DFF758BFF7560
:100043008850D29975816075A8827530007531002A
:10005300753508753605D220C221D222C223D22497
:10006300C225D226C227D228C229D22AC22BD22CF9
:10007300C22DD22EC22FD230D231D234C235D23693
:10008300C237D250C251D253D2A020A01230201F67
:10009300C22020210512039080151203B280102084
:1000A300200DD2202021051203AE80031203D1D2EA
:1000B300A120A11230221FC2222023051203D580C2
:1000C300151203F7801020220DD2222023051203DC
:1000D300F38003120416D2A220A21230241FC224DA
:1000E30020250512041A801512043C801020240DCB
:1000F300D224202505120438800312045BD2A320E6
:10010300A31230261FC22620270512045F80151272
:100113000481801020260DD22620270512047D801D
:10012300031204A0D2A420A41230281FC22820291D
:10013300051204A480151204C6801020280DD228AD
:100143002029051204C280031204E5D2A520A512BA
:10015300302A1FC22A202B051204E9801512050B31
:100163008010202A0DD22A202B05120507800312A6
:10017300052AD2A620A612302C1FC22C202D051230
:10018300052E80151205508010202C0DD22C202D09
:100193000512054C800312056FD2A720A712302E3B
:1001A3001FC22E202F05120573801512059580108E
:1001B300202E0DD22E202F0512059180031205B497
:1001C300D2B020B014303021C230B2312031051208
:1001D30005B880151205DA801020300DD230203199
:1001E300051205D680031205F8D2B220B2123034BC
:1001F3001FC2342035051205FC801512061E80101F
:1002030020340DD23420350512061A800312063D20
:10021300D2B320B31230361FC2362037051206413F
:100223008015120663801020360DD2362037051252
:10023300065F8003120683D2B420B41C7532071202
:100243000687120382D5320675320112068712031E
:1002530089D2B420B40280EDD2B520B51C75320723
:100263001206BB120382D532067532011206BB1287
:100273000389D2B520B50280EDD2B620B61C753203
:10028300071206EF120382D532067532011206EF0A
:10029300120389D2B620B60280EDD2B720B71C75FF
:1002A3003207120702120382D53206753201120792
:1002B30002120389D2B720B70280ED438701018B75
:1002C30002003332C0D0C0E0C083C082E530900961
:1002D3001593F535E53190097993F5363054037567
:1002E30035F62053037536FB305016C250D2517584
:1002F3003300753400A25392527580FF7590FE80CF
:100303002A205127B252A252400885358085369063
:1003130080067580FF7590FF0533E53390071593CD
:10032300F58CD082D083D0E0D0D032B252A25240EA
:100333000885358085369080067580FF7590FF05AA
:1003430034E534B4FF18C251A25392527580FF753D
:1003530090FF758CFFD082D083D0E0D0D032D29082
:1003630024FC4008C2907590FE7580FF9008159399
:10037300F58CD082D083D0E0D0D032323232327E8C
:1003830080DFFEDEFC227E60DFFEDEFC22D253D263
:10039300503099FDC2997599C03099FDC299E530E5
:1003A3007531002531F5991203822212038222C28C
:1003B30054C221C223C225C227C229C22BC22DC2C5
:1003C3002FC235C237D25075300012038222120376
:1003D3008222D253D2503099FDC2997599C0309977
:1003E300FDC299E5307531012531F5991203822259
:1003F30012038222C254C221C223C225C227C229A8
:10040300C22BC22DC22FC235C237D25075300A1249
:1004130003822212038222D253D2503099FDC29911
:100423007599C03099FDC299E5307531022531F5D2
:10043300991203822212038222C254C221C223C20E
:1004430025C227C229C22BC22DC22FC235C237D221
:10045300507530141203822212038222D253D250D7
:100463003099FDC2997599C03099FDC299E53075EF
:1004730031032531F5991203822212038222C254D9
:10048300C221C223C225C227C229C22BC22DC22F19
:10049300C235C237D25075301E1203822212038234
:1004A30022D253D2503099FDC2997599C03099FD2B
:1004B300C299E5307531042531F599120382221270
:1004C300038222C254C221C223C225C227C229C227
:1004D3002BC22DC22FC235C237D25075302812031A
:1004E300822212038222D253D2503099FDC29975CF
:1004F30099C03099FDC299E5307531052531F599DB
:100503001203822212038222C254C221C223C225B1
:10051300C227C229C22BC22DC22FC235C237D25025
:100523007530321203822212038222D253D2503008
:1005330099FDC2997599C03099FDC299E53075311D
:10054300062531F5991203822212038222C254C274
:1005530021C223C225C227C229C22BC22DC22FC248
:1005630035C237D25075303C1203822212038222E5
:10057300D253D2503099FDC2997599C03099FDC2BA
:1005830099E5307531072531F5991203822212035B
:100593008222C254C221C223C225C227C229C22B2E
:1005A300C22DC22FC235C237D250753046120382D4
:1005B3002212038222D254C253D250D221D223D246
:1005C30025D227D229D22BD22DD22FD235D23712F0
:1005D30003822212038222D254C253D250D221D296
:1005E30023D225D227D229D22BD22DD22FD235D224
:1005F300371203822212038222D253D2503099FD42
:10060300C2997599C03099FDC299E53075310825B5
:1006130031F5991203822212038222C254C221C2EB
:1006230023C225C227C229C22BC22DC22FC235C263
:1006330037D2507530501203822212038222D253D2
:10064300D2503099FDC2997599C03099FDC299E590
:10065300307531092531F599120382221203822262
:10066300C254C221C223C225C227C229C22BC22D12
:10067300C22FC235C237D25075305A12038222229A
:1006830012038222C254D253D250053174F625315B
:100693007012753100E530240AF530749C253070F2
:1006A300037530003099FDC2997599C03099FDC228
:1006B30099E5302531F59922C254D253D2501531E0
:1006C300740125317012753109E53024F6F5307463
:1006D3000A2530700375305A3099FDC2997599C057
:1006E3003099FDC299E5302531F59922C253D25094
:1006F300E530240AF530946460012275300022C28B
:1007030053D250E53024F6F53094F660012275306B
:100713005A22FFE0FFE0FFE0FFE0FFE0FEE1FEE141
:10072300FEE1FEE1FEE1FDE2FDE2FDE2FDE2FDE2CE
:10073300FCE3FCE3FCE3FCE3FCE3FBE4FBE4FBE4BE
:10074300FBE4FBE4FAE5FAE5FAE5FAE5FAE5F9E6AE
:10075300F9E6F9E6F9E6F9E6F8E7F8E7F8E7F8E79E
:10076300F8E7F7E8F7E8F7E8F7E8F7E8F6E9F6E98E
:10077300F6E9F6E9F6E9F5EAF5EAF5EAF5EAF5EA7E
:10078300F4EBF4EBF4EBF4EBF4EBF3ECF3ECF3EC6E
:10079300F3ECF3ECF2EDF2EDF2EDF2EDF2EDF1EE5E
:1007A300F1EEF1EEF1EEF1EEF0EFF0EFF0EFF0EF4E
:1007B300F0EFF0EFF0EFF0EFF0EFF0EFF0EFF0EF3E
:1007C300F0EFF0EFF0EFF0EFF0EFF0EFF0EFF0EF2E
:1007D300F0EFF0EFF0EFF1EEF1EEF2EDF2EDF3EC1E
:1007E300F3ECF4EBF4EBF5EAF5EAF6E9F6E9F7E80E
:1007F300F7E8F8E7F8E7F9E6F9E6FAE5FAE5FBE4FE
:10080300FBE4FCE3FCE3FDE2FDE2FEE1FEE1FFE0ED
:10081300FFE0E0FFE3FCE6F9E9F6ECF3EFF0F2EDDD
:10082300F5EAF8E7FBE4FEE1FFE0FFE0FFE0FFE0CD
:10083300FFE0FEE1FEE1FEE1FEE1FEE1FDE2FDE2BD
:10084300FDE2FDE2FDE2FCE3FCE3FCE3FCE3FCE3AD
:10085300FBE4FBE4FBE4FBE4FBE4FAE5FAE5FAE59D
:10086300FAE5FAE5F9E6F9E6F9E6F9E6F9E6F8E78D
:10087300F8E7F8E7F8E7F8E7F7E8F7E8F7E8F7E87D
:10088300F7E8F6E9F6E9F6E9F6E9F6E9F5EAF5EA6D
:10089300F5EAF5EAF5EAF4EBF4EBF4EBF4EBF4EB5D
:1008A300F3ECF3ECF3ECF3ECF3ECF2EDF2EDF2ED4D
:1008B300F2EDF2EDF1EEF1EEF1EEF1EEF1EEF0EF3D
:1008C300F0EFF0EFF0EFF0EFF0EFF0EFF0EFF0EF2D
:1008D300F0EFF0EFF0EFF1EEF1EEF2EDF2EDF3EC1D
:1008E300F3ECF4EBF4EBF5EAF5EAF6E9F6E9F7E80D
:1008F300F7E8F8E7F8E7F9E6F9E6FAE5FAE5FBE4FD
:10090300FBE4FCE3FCE3FDE2FDE2FEE1FEE1FFE0EC
:10091300FFE008000000000000000000DC00000011
:100923000000000000003000000000000000000094
:1009330090000000000000000000C4000000000060
:100943000000000082000000000000000000020020
:100953000000000000000000D800000000000000BC
:100963000000000000000000000000008000000004
:1009730000000000000005DD83915931219D011124
:10098300204D757A796B616E7420322076312E306A
:1009930020323030362D31302D3232202863294138
:1009A30064616D20536D69616C656B206A616E6B68
:1009B3006F6D757A796B616E744077702E706C20F1
:1009C3007777772E736D69616C656B2E7072762EF7
:1009D300706C2057737A656C6B69652070726177F0
:1009E30061207A617374727A657A6F6E652E204A1C
:1009F300616B69656B6F6C7769656B207A61737482
:100A03006F736F77616E6961206B6F6D6572637968
:100A13006A6E65206B6F6475206E6965646F7A77A3
:100A23006F6C6F6E652E20416C6C20526967687421
:100A3300732052657365727665642E204672656510
:100A430020666F72206E6F6E20636F6D6D657263CB
:0A0A530069616C206F6E6C792E2033
:00000001FF
